:020000040000FA
:04080000E4EF04F02D
:1008100003B23DEF04F0F2B458EF04F09EB060EF85
:1008200004F09EB268EF04F0F2A81AEF04F0F2B2FE
:100830001CEF04F0C2EF04F0CD90F29207BC078EDB
:10084000078C9EA029EF04F00101463F29EF04F038
:10085000472B07AE34EF04F0CECF4EF1CFCF4FF1A0
:1008600046C150F147C151F1CF6ACE6A0101466BD2
:10087000476B9E90CD80C2EF04F00392030103EE1C
:1008800000F080517F0BE92604C0EFFF802B8151DF
:10089000805D700BD8A48B8200008051815D700B4D
:1008A000D8A48B9281518019D8B40790C2EF04F07C
:1008B000F2940101383FC2EF04F0392BC2EF04F08B
:1008C0009E900101463FC2EF04F0472BC2EF04F0B7
:1008D0009E92C3CF48F1C4CF49F1C28207B485EFDD
:1008E00004F03AC13EF13BC13FF13CC140F13DC192
:1008F00041F14EC152F14FC153F150C154F151C1B8
:1009000055F148C14AF149C14BF10201002FC2EF34
:1009100004F03C0E006FD57ED5BE32D0D6CF3AF172
:10092000D7CF3BF138C13CF1E86AE8CF3DF1010196
:1009300047A7A6EF04F0079C079E0101000E4E6F2B
:10094000600E4F6F3D0E506F080E516F01013ABFA0
:10095000B6EF04F03B67B6EF04F03C67B6EF04F087
:100960003D67B6EF04F0F288BBEF04F0F2984E6BEF
:100970004F6B506B516BD76AD66A0101386B396B7C
:10098000C2EF04F002C0E0FF005001C0D8FF100029
:10099000A6B2C8EF04F00CC0A9FF0BC0A8FFA69E2A
:1009A000A69CA684F29E550EA76EAA0EA76EA682DE
:1009B000F28EA694A6B2DAEF04F01200A96EA69EFB
:1009C000A69CA680A8501200076A0F010E0EC16EE9
:1009D000800EC06E030EC26E0F01896A110E926EF8
:1009E000080E8A6EF10E936E8B6A800E946EF18EF5
:1009F0000F01280ED56EF28AB00ECD6E9D800101DA
:100A00004E6B4F6B506B516B526B536B546B556B02
:100A1000566B576B586B596B079C079E760ECA6EC8
:100A20009D8202013C0E006FCC6A240EAC6E040164
:100A3000806B816B0F01900EAB6E0F019D8A0301DD
:100A4000806B816BA26B8B9207900001F28EF28C0F
:100A500007B088EF0CF08B740301805181197F0B74
:100A6000D8B488EF0CF013EE00F081517F0BE12633
:100A7000812BE7CFE8FFE00BD8B488EF0CF023EE32
:100A800082F0A2511F0BD926E7CFDFFFA22BDF5048
:100A9000780AD8A488EF0CF007808251720AD8B483
:100AA00008EF07F08251630AD8B448EF09F0825189
:100AB000690AD8B47BEF05F082517A0AD8B48EEF78
:100AC00006F07DEF09F0040114EE00F080517F0B79
:100AD000E12682C4E7FF802B12000D0E826F63ECCB
:100AE00005F00A0E826F63EC05F01200040E826FAF
:100AF00063EC05F012000401690E826F63EC05F0EF
:100B000004012C0E826F63EC05F00101040E006FEE
:100B1000000E016F000E026F000E036F17EC0FF056
:100B200020C182F40401300E822763EC05F021C15C
:100B300082F40401300E822763EC05F022C182F4B6
:100B40000401300E822763EC05F023C182F4040116
:100B5000300E822763EC05F024C182F40401300ECC
:100B6000822763EC05F025C182F40401300E822750
:100B700063EC05F026C182F40401300E822763EC99
:100B800005F027C182F40401300E822763EC05F0E2
:100B900004012C0E826F63EC05F00101030E006F5F
:100BA000000E016F000E026F000E036F17EC0FF0C6
:100BB00020C182F40401300E822763EC05F021C1CC
:100BC00082F40401300E822763EC05F022C182F426
:100BD0000401300E822763EC05F023C182F4040186
:100BE000300E822763EC05F024C182F40401300E3C
:100BF000822763EC05F025C182F40401300E8227C0
:100C000063EC05F026C182F40401300E822763EC08
:100C100005F027C182F40401300E822763EC05F051
:100C200004012C0E826F63EC05F001010C0E006FC5
:100C3000000E016F000E026F000E036F17EC0FF035
:100C400020C182F40401300E822763EC05F021C13B
:100C500082F40401300E822763EC05F022C182F495
:100C60000401300E822763EC05F023C182F40401F5
:100C7000300E822763EC05F024C182F40401300EAB
:100C8000822763EC05F025C182F40401300E82272F
:100C900063EC05F026C182F40401300E822763EC78
:100CA00005F027C182F40401300E822763EC05F0C1
:100CB00004012C0E826F63EC05F0200EF86EF76ACB
:100CC000F66A04010900F5CF82F463EC05F009002F
:100CD000F5CF82F463EC05F00900F5CF82F463EC04
:100CE00005F00900F5CF82F463EC05F00900F5CFBB
:100CF00082F463EC05F00900F5CF82F463EC05F0B3
:100D00000900F5CF82F463EC05F00900F5CF82F419
:100D100063EC05F06DEC05F07DEF09F08351630A9B
:100D2000D8A47DEF09F08451610AD8A47DEF09F0C1
:100D300085516C0AD8A47DEF09F08651410A42E042
:100D40008651440A1BE08651420AD8B4F5EF06F0FA
:100D50008651350AD8B406EF0BF08651360AD8B45E
:100D60005AEF0BF08651370AD8B4C2EF0BF0865118
:100D7000380AD8B420EF0CF07DEF09F00798079AF5
:100D800004017A0E826F63EC05F00401780E826F25
:100D900063EC05F00401640E826F63EC05F081A83A
:100DA000D9EF06F00401550E826F63EC05F0DEEF1B
:100DB00006F004014C0E826F63EC05F06DEC05F05B
:100DC0007DEF09F00788079A04017A0E826F63ECC1
:100DD00005F00401410E826F63EC05F00401610E21
:100DE000826F63EC05F0CFEF06F00798078A0401E5
:100DF0007A0E826F63EC05F00401420E826F63ECA1
:100E000005F00401610E826F63EC05F0CFEF06F090
:100E10000401720E826F63EC05F004012C0E826FE8
:100E200063EC05F0078452C156F153C157F154C128
:100E300058F155C159F13EC142F13FC143F140C1A2
:100E400044F141C145F14AC14CF14BC14DF1079408
:100E50000101620E046F010E056F000E066F000E99
:100E6000076F56C100F157C101F158C102F159C1D4
:100E700003F17DEC0EF003BF85EF07F00E0EDEEC04
:100E800004F0E8CF0CF10F0EDEEC04F0E8CF0DF12A
:100E9000100EDEEC04F0E8CF0EF1110EDEEC04F0E3
:100EA000E8CF0FF1C6EC0DF056C104F157C105F1C2
:100EB00058C106F159C107F17DEC0EF007828AECAA
:100EC0000DF0C6EC0DF007928AEC0DF056C100F162
:100ED00057C101F158C102F159C103F107928AECDF
:100EE0000DF0CC0E046FE00E056F870E066F050E39
:100EF000076F7DEC0EF000C10CF101C10DF102C1D4
:100F00000EF103C10FF1BEEF07F00101800E006F7B
:100F10001A0E016F060E026F000E036F42C104F13C
:100F200043C105F144C106F145C107F17DEC0EF066
:100F300003AF9FEF07F074EC0FF0D1EF07F00E0E48
:100F4000DEEC04F0E8CF0CF10F0EDEEC04F0E8CF9D
:100F50000DF1100EDEEC04F0E8CF0EF1110EDEEC18
:100F600004F0E8CF0FF142C100F143C101F144C1E7
:100F700002F145C103F107828AEC0DF00CC100F1CA
:100F80000DC101F10EC102F10FC103F10101000E0B
:100F9000046F000E056F010E066F000E076FABECBD
:100FA0000EF017EC0FF01D67DBEF07F00401200EC9
:100FB000826FDEEF07F004012D0E826F63EC05F007
:100FC00024C182F40401300E822763EC05F025C1B0
:100FD00082F40401300E822763EC05F004012E0E2A
:100FE000826F63EC05F026C182F40401300E822783
:100FF00063EC05F027C182F40401300E822763EC14
:1010000005F004016D0E826F63EC05F004012C0EF7
:10101000826F63EC05F042C100F143C101F144C1AC
:1010200002F145C103F1010117EC0FF01EC182F47A
:101030000401300E822763EC05F01FC182F4040125
:10104000300E822763EC05F020C182F40401300EDB
:10105000822763EC05F021C182F40401300E82275F
:1010600063EC05F022C182F40401300E822763ECA8
:1010700005F023C182F40401300E822763EC05F0F1
:1010800024C182F40401300E822763EC05F025C1EF
:1010900082F40401300E822763EC05F026C182F44D
:1010A0000401300E822763EC05F027C182F40401AD
:1010B000300E822763EC05F00401480E826F63EC6A
:1010C00005F004017A0E826F63EC05F004012C0E2A
:1010D000826F63EC05F056C100F157C101F158C1B0
:1010E00002F159C103F1010117EC0FF01EC182F4A6
:1010F0000401300E822763EC05F01FC182F4040165
:10110000300E822763EC05F020C182F40401300E1A
:10111000822763EC05F021C182F40401300E82279E
:1011200063EC05F022C182F40401300E822763ECE7
:1011300005F023C182F40401300E822763EC05F030
:1011400024C182F40401300E822763EC05F025C12E
:1011500082F40401300E822763EC05F026C182F48C
:101160000401300E822763EC05F027C182F40401EC
:10117000300E822763EC05F00401630E826F63EC8E
:1011800005F004012C0E826F63EC05F056C100F1EE
:1011900057C101F158C102F159C103F101010A0E11
:1011A000046F000E056F000E066F000E076F8CECCB
:1011B0000EF0000E046F120E056F000E066F000E8B
:1011C000076FABEC0EF017EC0FF01EC182F40401B8
:1011D000300E822763EC05F01FC182F40401300E4B
:1011E000822763EC05F020C182F40401300E8227CF
:1011F00063EC05F021C182F40401300E822763EC18
:1012000005F022C182F40401300E822763EC05F060
:1012100023C182F40401300E822763EC05F024C15F
:1012200082F40401300E822763EC05F004012E0ED7
:10123000826F63EC05F025C182F40401300E822731
:1012400063EC05F026C182F40401300E822763ECC2
:1012500005F027C182F40401300E822763EC05F00B
:101260000401730E826F63EC05F004012C0E826F93
:1012700063EC05F074EC0FF04CC100F14DC101F1CD
:10128000A6EC0AF06DEC05F076EC05F07DEF09F0C8
:101290000401630E826F63EC05F004012C0E826F73
:1012A00063EC05F082EC09F004012C0E826F63EC14
:1012B00005F0F5EC09F004012C0E826F63EC05F0EB
:1012C00071EC0AF004012C0E826F63EC05F0010151
:1012D000F80E006FCD0E016F660E026F030E036FE6
:1012E00097EC09F004012C0E826F63EC05F087EC9B
:1012F0000AF06DEC05F07DEF09F00301A26B079099
:1013000088EF0CF0D8900E0EDEEC04F0E8CF00F180
:101310000F0EDEEC04F0E8CF01F1100EDEEC04F06D
:10132000E8CF02F1110EDEEC04F0E8CF03F1010189
:10133000000E046F000E056F010E066F000E076FA2
:10134000ABEC0EF017EC0FF01EC182F40401300E6E
:10135000822763EC05F01FC182F40401300E82275E
:1013600063EC05F020C182F40401300E822763ECA7
:1013700005F021C182F40401300E822763EC05F0F0
:1013800022C182F40401300E822763EC05F023C1F0
:1013900082F40401300E822763EC05F024C182F44C
:1013A0000401300E822763EC05F025C182F40401AC
:1013B000300E822763EC05F004012E0E826F63EC81
:1013C00005F026C182F40401300E822763EC05F09B
:1013D00027C182F40401300E822763EC05F004017A
:1013E0006D0E826F63EC05F01200120EDEEC04F05D
:1013F000E8CF00F1130EDEEC04F0E8CF01F1140E9B
:10140000DEEC04F0E8CF02F1150EDEEC04F0E8CFDC
:1014100003F101010A0E046F000E056F000E066F46
:10142000000E076F8CEC0EF0000E046F120E056FAD
:10143000000E066F000E076FABEC0EF017EC0FF00E
:101440001EC182F40401300E822763EC05F01FC137
:1014500082F40401300E822763EC05F020C182F48F
:101460000401300E822763EC05F021C182F40401EF
:10147000300E822763EC05F022C182F40401300EA5
:10148000822763EC05F023C182F40401300E822729
:1014900063EC05F024C182F40401300E822763EC72
:1014A00005F004012E0E826F63EC05F025C182F475
:1014B0000401300E822763EC05F026C182F404019A
:1014C000300E822763EC05F027C182F40401300E50
:1014D000822763EC05F00401730E826F63EC05F064
:1014E00012000A0EDEEC04F0E8CF00F10B0EDEEC89
:1014F00004F0E8CF01F10C0EDEEC04F0E8CF02F1CD
:101500000D0EDEEC04F0E8CF03F1A6EF0AF0060EB4
:10151000DEEC04F0E8CF00F1070EDEEC04F0E8CFDB
:1015200001F1080EDEEC04F0E8CF02F1090EDEEC6A
:1015300004F0E8CF03F1A6EF0AF0010174EC0FF01C
:1015400007844AC100F14BC101F107940101E80E83
:10155000046F800E056F000E066F000E076F8CEC97
:101560000EF0000E046F040E056F000E066F000EE5
:10157000076FABEC0EF0880E046F130E056F000EB4
:10158000066F000E076F7DEC0EF00A0E046F000E62
:10159000056F000E066F000E076FABEC0EF017EC38
:1015A0000FF001011D67DAEF0AF00401200E826FCF
:1015B000DDEF0AF004012D0E826F63EC05F024C10B
:1015C00082F40401300E822763EC05F025C182F419
:1015D0000401300E822763EC05F026C182F4040179
:1015E000300E822763EC05F004012E0E826F63EC4F
:1015F00005F027C182F40401300E822763EC05F068
:101600000401430E826F63EC05F0120087C31EF1E4
:1016100088C31FF189C320F18AC321F18BC322F152
:101620008CC323F18DC324F18EC325F190C326F121
:1016300091C327F10101C1EC0FF039EC0FF001016A
:10164000000E046F000E056F010E066F000E076F8F
:101650008CEC0EF00E0E0C6E00C10BF0C8EC04F01A
:101660000F0E0C6E01C10BF0C8EC04F0100E0C6EE6
:1016700002C10BF0C8EC04F0110E0C6E03C10BF0AC
:10168000C8EC04F004017A0E826F63EC05F00401EB
:101690002C0E826F63EC05F00401350E826F63EC53
:1016A00005F004012C0E826F63EC05F082EC09F06A
:1016B000DEEF06F087C31EF188C31FF189C320F156
:1016C0008AC321F18BC322F18CC323F18DC324F192
:1016D0008EC325F190C326F191C327F10101C1EC1E
:1016E0000FF039EC0FF0880E046F130E056F000E2B
:1016F000066F000E076F81EC0EF0000E046F040EF3
:10170000056F000E066F000E076F8CEC0EF00101E6
:10171000E80E046F800E056F000E066F000E076F57
:10172000ABEC0EF00A0E0C6E00C10BF0C8EC04F02E
:101730000B0E0C6E01C10BF0C8EC04F00C0E0C6E1D
:1017400002C10BF0C8EC04F00D0E0C6E03C10BF0DF
:10175000C8EC04F004017A0E826F63EC05F004011A
:101760002C0E826F63EC05F00401360E826F63EC81
:1017700005F004012C0E826F63EC05F071EC0AF0A9
:10178000DEEF06F087C31EF188C31FF189C320F185
:101790008AC321F18BC322F18CC323F18DC324F1C1
:1017A0008FC325F190C326F191C327F10101C1EC4C
:1017B0000FF039EC0FF0000E046F120E056F000EE3
:1017C000066F000E076F8CEC0EF001010A0E046F1D
:1017D000000E056F000E066F000E076FABEC0EF0EB
:1017E000120E0C6E00C10BF0C8EC04F0130E0C6E60
:1017F00001C10BF0C8EC04F0140E0C6E02C10BF02A
:10180000C8EC04F0150E0C6E03C10BF0C8EC04F02C
:1018100004017A0E826F63EC05F004012C0E826FD6
:1018200063EC05F00401370E826F63EC05F00401F0
:101830002C0E826F63EC05F0F5EC09F0DEEF06F09C
:1018400087C31EF188C31FF189C320F18AC321F128
:101850008BC322F18CC323F18DC324F18EC325F1F8
:1018600090C326F191C327F10101C1EC0FF039ECCF
:101870000FF0880E046F130E056F000E066F000E3A
:10188000076F81EC0EF0000E046F040E056F000E62
:10189000066F000E076F8CEC0EF00101E80E046F6E
:1018A000800E056F000E066F000E076FABEC0EF09A
:1018B000060E0C6E00C10BF0C8EC04F0070E0C6EA7
:1018C00001C10BF0C8EC04F0080E0C6E02C10BF065
:1018D000C8EC04F0090E0C6E03C10BF0C8EC04F068
:1018E00004017A0E826F63EC05F004012C0E826F06
:1018F00063EC05F00401380E826F63EC05F004011F
:101900002C0E826F63EC05F087EC0AF0DEEF06F038
:1019100081A846EF0DF007A8FFEF0CF00101800E43
:10192000006F1A0E016F060E026F000E036F3EC1AC
:1019300004F13FC105F140C106F141C107F17DEC61
:101940000EF003BF46EF0DF084EC0DF03EC100F148
:101950003FC101F140C102F141C103F107828AECAC
:101960000DF00CC104F10DC105F10EC106F10FC15E
:1019700007F1F80E006FCD0E016F660E026F030EB9
:10198000036F7DEC0EF00E0E0C6E00C10BF0C8EC78
:1019900004F00F0E0C6E01C10BF0C8EC04F0100E39
:1019A0000C6E02C10BF0C8EC04F0110E0C6E03C1FA
:1019B0000BF0C8EC04F00784010174EC0FF04AC18D
:1019C00000F14BC101F107940A0E0C6E00C10BF03F
:1019D000C8EC04F00B0E0C6E01C10BF0C8EC04F067
:1019E0000C0E0C6E02C10BF0C8EC04F00D0E0C6E68
:1019F00003C10BF0C8EC04F0079846EF0DF007AAFE
:101A000046EF0DF00784010174EC0FF04AC100F1BC
:101A10004BC101F10794060E0C6E00C10BF0C8EC2F
:101A200004F0070E0C6E01C10BF0C8EC04F0080EB8
:101A30000C6E02C10BF0C8EC04F0090E0C6E03C171
:101A40000BF0C8EC04F0078452C100F153C101F15E
:101A500054C102F155C103F10794120E0C6E00C17E
:101A60000BF0C8EC04F0130E0C6E01C10BF0C8ECC7
:101A700004F0140E0C6E02C10BF0C8EC04F0150E4D
:101A80000C6E03C10BF0C8EC04F0079A04018051FE
:101A900081197F0B0BE09EA809D014EE00F0815154
:101AA0007F0BE126E750812B0F01AD6E28EF05F08B
:101AB0000CC100F10DC101F10EC102F10FC103F122
:101AC000000E046F000E056F010E066F000E076F0B
:101AD000ABEC0EF01DA183EF0DF01451D8B483EFE1
:101AE0000DF00CC100F10DC101F10EC102F10FC1E9
:101AF00003F1000E046F000E056F0A0E066F000E54
:101B0000076FABEC0EF0120001010C6B0D6B0E6B4E
:101B10000F6B12000101005305E1015303E1025371
:101B200001E1002B4DEC0EF074EC0FF02C51006F26
:101B30002D51016F420E046F4B0E056F000E066FA4
:101B4000000E076F8CEC0EF000C104F101C105F12D
:101B500002C106F103C107F10CC100F10DC101F191
:101B60000EC102F10FC103F107B2BBEF0DF081EC22
:101B70000EF0BDEF0DF07DEC0EF000C10CF101C1D7
:101B80000DF102C10EF103C10FF1120074EC0FF060
:101B90004CC100F14DC101F1060EDEEC04F0E8CFBE
:101BA00004F1070EDEEC04F0E8CF05F1080EDEECE0
:101BB00004F0E8CF06F1090EDEEC04F0E8CF07F1FF
:101BC0007DEC0EF000C118F101C119F102C11AF14A
:101BD00003C11BF1290E046F000E056F000E066F86
:101BE000000E076F8CEC0EF0EE0E046F430E056FC7
:101BF000000E066F000E076F81EC0EF018C104F1A5
:101C000019C105F11AC106F11BC107F18CEC0EF0E8
:101C100000C110F101C111F102C112F103C113F1B0
:101C2000120EDEEC04F0E8CF04F1130EDEEC04F04B
:101C3000E8CF05F1140EDEEC04F0E8CF06F1150E46
:101C4000DEEC04F0E8CF07F10D0E006F000E016F1F
:101C5000000E026F000E036F8CEC0EF0180E046F76
:101C6000000E056F000E066F000E076FABEC0EF056
:101C700010C104F111C105F112C106F113C107F140
:101C800081EC0EF06A0E046F2A0E056F000E066FCF
:101C9000000E076F7DEC0EF01200BF0EFA6E200EE4
:101CA0002D6F2C6BD8900037013702370337D8B02F
:101CB0005EEF0EF02D2F53EF0EF02C072D07035380
:101CC000D8B412000331070B8009326F03390F0BB0
:101CD000010F2C6F80EC5FF0336F2C0580EC5FF010
:101CE000335D335F2C6B3233D8B02C272C3332A9C1
:101CF00073EF0EF033512C27120099EC0FF0D8B08F
:101D0000120003510719286F5CEC0FF0D8900751AF
:101D1000031928AF800F1200286B80EC0FF0D8A0B9
:101D200096EC0FF0D8B012006BEC0FF074EC0FF0E3
:101D30001F0E296FACEC0FF00B35D8B05CEC0FF038
:101D4000D8A00335D8B01200292F9AEF0EF028B191
:101D500083EC0FF01200286B0451051106110711D6
:101D60000008D8A080EC0FF0D8A096EC0FF0D8B007
:101D70001200086B096B0A6B0B6BACEC0FF01F0EBB
:101D8000296FACEC0FF007510B5DD8A4D4EF0EF027
:101D900006510A5DD8A4D4EF0EF00551095DD8A410
:101DA000D4EF0EF00451085DD8A0E7EF0EF0045117
:101DB000085F0551D8A0053D095F0651D8A0063D32
:101DC0000A5F0751D8A0073D0B5FD8900081292FEB
:101DD000C1EF0EF028B183EC0FF0286B80EC0FF010
:101DE000D890B0EC0FF007510B5DD8A404EF0FF0C2
:101DF00006510A5DD8A404EF0FF00551095DD8A47F
:101E000004EF0FF00451085DD8A013EF0FF0003F6E
:101E100013EF0FF0013F13EF0FF0023F13EF0FF03E
:101E2000032BD8B4120028B183EC0FF0120001018B
:101E3000286B80EC0FF0D8B01200B5EC0FF0200E3C
:101E4000296F003701370237033711EE27F00A0EEA
:101E50002A6FE7360A0EE75CD8B0E76EE5522A2F04
:101E600029EF0FF0292F21EF0FF028B11D81D89015
:101E7000120001010A0E286F200E296F11EE1DF0CD
:101E800028512A6F0A0ED890E652D8B0E726E732DA
:101E90002A2F44EF0FF00333023301330033292F8D
:101EA0003EEF0FF0E750FF0FD8A00335D8B0120077
:101EB0001DB183EC0FF01200045100270551D8B07A
:101EC000053D01270651D8B0063D02270751D8B07D
:101ED000073D032712000051086F0151096F02519D
:101EE0000A6F03510B6F12000101006B016B026B53
:101EF000036B12000101046B056B066B076B12008C
:101F00000335D8A012000351800B001F011F021FD0
:101F1000031F003F93EF0FF0013F93EF0FF0023FDD
:101F200093EF0FF0032B282B032512000735D8A0C1
:101F300012000751800B041F051F061F071F043FD7
:101F4000A9EF0FF0053FA9EF0FF0063FA9EF0FF043
:101F5000072B282B072512000037013702370337DC
:101F6000083709370A370B3712001D6B1E6B1F6BC2
:101F7000206B216B226B236B246B256B266B276BED
:101F800012001E510F0B1E6F1F510F0B1F6F2051A0
:101F90000F0B206F21510F0B216F22510F0B226F5E
:101FA00023510F0B236F24510F0B246F25510F0B5F
:101FB000256F26510F0B266F27510F0B276F12002D
:10BF0000E844F926000C160C2B0C3F0C520C640C68
:10BF1000760C860C960CA50CB30CC10CCF0CDC0C6B
:06BF2000E80CF40C000C1B
:00000001FF
